:020000040100F9
:10000000882900205D010001E90400015D04000170
:1000100000000000000000000000000000000000E0
:10002000000000000000000000000000F1070001D7
:1000300000000000000000001B010001F5070001A6
:100040006F0100016F0100016F0100016F010001EC
:100050006F0100016F0100016F0100016F010001DC
:100060006F0100016F0100016F0100016F010001CC
:100070006F0100016F0100016F0100016F010001BC
:100080006F0100016F0100016F0100016F010001AC
:100090006F0100016F0100016F0100016F0100019C
:1000A0006F0100016F0100016F0100016F0100018C
:1000B0006F0100016F0100016F0100016F0100017C
:1000C0000348854600F0C2F800480047150E0001BD
:1000D0008829002040BA7047C0BA70470138FDD166
:1000E00070470000084B19680868203080F30988C1
:1000F000022080F31488BFF36F8F3FBCAE4608BC6C
:1001000004BC62B61847000004000020EFF3108022
:1001100072B6704780F310887047EFF309800E4B7A
:100120001A6820381060F0C044464D4656465F4677
:10013000F0C008B572B601F0B9FB62B60CBC11682C
:1001400008681030F0C8A046A946B246BB4680F306
:1001500009882038F0C81847040000200448804768
:1001600004480047FEE7FEE7FEE7FEE7FEE7FEE79E
:1001700029080001C100000130B50B4601460020EE
:100180002022012409E00D46D5409D4205D31D469D
:100190009540491B2546954040191546521E002D95
:1001A000F1DC30BD03460B439B0703D009E008C9CF
:1001B000121F08C0042AFAD203E00B780370401C17
:1001C000491C521EF9D27047D2B201E00270401CA5
:1001D000491EFBD270470022F6E710B513460A46C7
:1001E00004461946FFF7F0FF204610BDF0B51FB4D6
:1001F0000646002082B005464024019100901BE095
:10020000019922460F46304600F042F8049A059BB9
:10021000801A994110D310461946224600F028F85A
:10022000361A8F410197224601200021009F00F0DD
:100230001FF838184D4100902046641E0028DFDC6E
:10024000019B00982946324607B0F0BD064C0125B7
:10025000064E05E0E36807CC2B430C3C984710346E
:10026000B442F7D3FFF730FFEC2200010C2300016A
:1002700010B5202A04DB0146203A9140002010BD31
:10028000914020239C1A0346E3401943904010BD3F
:1002900010B5202A04DB0846203AD040002110BDCA
:1002A0000B46D340D0402024A21A9140084319465F
:1002B00010BD00001CB5002208210A2001F052FBED
:1002C000104908600020022103468022009101901D
:1002D0000DA10F4801F032FD0020022103468022CB
:1002E000009101900BA10D4801F028FD0020032191
:1002F0000346FF2201320091019009A10A4801F052
:100300001DFD1CBD5C0000204C4544310000000078
:10031000610400014C45443200000000A5040001C6
:100320005052494E54000000B905000170B5034613
:100330000A4600210024002076E001268E40156840
:1003400035402C46002C6ED05568022D02D05568E1
:10035000122D20D108250D40002D0ED0586A4D07D2
:10036000EE0E0F25B5400646AE4330464E07F60E5C
:100370005569B540284358620DE0186A4D07EE0EE6
:100380000F25B5400646AE4330464E07F60E55697A
:10039000B540284318625568012D08D05568112DC5
:1003A00005D05568022D02D05568122D0BD1586822
:1003B00001258D400646AE4330461579ED06ED0F1A
:1003C0008D402843586018684E000325B540064606
:1003D000AE4330461579AD07AD0F4E00B54028430A
:1003E0001860D8684E000325B5400646AE43304637
:1003F0004E009568B5402843D860986801258D4027
:100400000646AE433046D5688D4028439860D86A8A
:100410004E000125B5400646AE4330464E001569F4
:10042000B5402843D862491C1568CD40002D84D1C1
:1004300070BD0000054901600F214161002141604C
:1004400081600121C160002101617047FF3F000010
:100450008162704742694A404261704700BFFEE7CF
:100460001CB50D4903C90191009000BF01210B4843
:1004700000F04AFC0120694608700198401C019078
:1004800000231A460648006801F0D5FAFF20F5302F
:1004900001F084F9EAE70000DC220001000C0140D1
:1004A0005C0000201CB50D4903C90191009000BFFC
:1004B00040210B4800F028FC022069460870019892
:1004C000401C019000231A460648006801F0B3FA68
:1004D0007D20C00001F062F9EAE70000E42200019B
:1004E000000801405C00002070470000F7B5D4B060
:1004F00004460E4600205390052052900025002708
:1005000000BFEFF310800090FF21453101A8FFF7F5
:1005100062FE01F067F805462448854218D10120A3
:100520000003844202D1002053902AE001204003BE
:10053000844202D14011539023E0032000038442FF
:1005400003D10120400253901BE0529857B0F0BDF8
:100550001748854213D101200003844201D15390F2
:100560000FE001204003844201D1539009E00320B1
:100570000003844201D1539003E05298E6E7529879
:10058000E4E705AF0137FF2241320A4901A8FFF72E
:1005900009FE012000F07DFA3146569A5398B8477B
:1005A0005290009800F075FA5298CFE7C4401300BB
:1005B00085601300F82000011CB500BF0022D24363
:1005C00069460648006801F0E3FA0128F6D168465A
:1005D000017803A0019A00F03DFAEFE75C000020EB
:1005E0004C4544257520746F67676C65642C2063E7
:1005F0006F756E74203D20256C750A00002905D0AA
:10060000054A92690243044B9A6104E0024A9269E6
:100610008243014B9A6170470010024010B50021DF
:100620000022214B5B68042423401946002902D094
:10063000042906D102E01D4B036005E01C4B03605A
:1006400002E01A4B036000BF00BF174B5B68302409
:10065000234019460909174B5A5C0368D34043608D
:10066000114B5B680724240223401946090A124BE8
:100670005A5C4368D34083600B4B5B68E4002340C3
:100680001946C90A0C4B5A5C4368D340C360064BF9
:10069000DB6A10242340002B02D0084B036102E0E8
:1006A0007D23DB03036110BD001002400090D003E6
:1006B0000048E801D8220001D022000100093D00D5
:1006C000F1B58AB0002009907D20C0000890012576
:1006D000AD020027002007907F20069040240026CE
:1006E00000200590039020010290002001903E49D7
:1006F0000A98884206D83D480068610288433B4911
:10070000086006E0394800680121C90308433749F9
:1007100008607D21C9000A98FFF72EFD7D21C900E0
:100720000090FFF729FD450100BF304800687F2198
:100730000902884301902002019908432B4908606F
:100740000520FFF7CBFC10E00120FFF7C7FC27488E
:10075000406B02210840002800D007E00598411CAA
:1007600005910899884200D900E0EDE700BF1F48D5
:10077000C06B86B2AE4201D9771B00E0AF1B029876
:10078000874203D2E0B20390B8B20290AE4201D3E6
:10079000069400E00794069907984018C005000EDB
:1007A00004900498A04200D103E0049C0998874279
:1007B000BBD800BF0D4800687F2109028843019023
:1007C00003980002019908430849086008464068F8
:1007D00040084000486000BF0448406804210840C9
:1007E0000028F9D10BB0F0BD0090D00300100240FA
:1007F0007047000010B5FFF789FC044601F0DEFAEF
:10080000002803D001200007024948602046FFF776
:1008100081FC10BD00ED00E001480249086070470E
:100820000090D0030000002010B53E48C0690121AF
:10083000090708433B49C861812000063A4908631B
:100840003A4848613A4808623A48006803218903F7
:100850008843384908603421374800F073F8364837
:100860000069401C002803D033480069002817D1D4
:100870002C4840680121090408432A494860084679
:1008800040680721090288432649486008464068B5
:1008900009150843234948602848FFF711FF3FE046
:1008A000214880694409640123480078C006C00ECD
:1008B00004431D4884611B4800680121C903884323
:1008C00018490860084600687F21090288430446E9
:1008D0001948006900022043124908600846406830
:1008E0000121090408430F49486008464068072170
:1008F000090288430B4948600846406809150843C7
:10090000084948600846006A0D49084005490862E0
:100910000846006A0849C968090208430149086293
:1009200010BD000000100240007000400F080000E1
:100930001800020000100140640000200090D00365
:10094000FF00F8FF70B504460D462A4621460120F7
:100950000003FFF7CBFD70BD002905D0828901237C
:100960005B031A43828103E08289024B1A40828131
:1009700070470000FFDF00000246002001235B02F9
:10098000994200D100BF13880B40002B01D00120F9
:1009900000E0002070470000F0B589B005460E4623
:1009A00000240020089000BF00BF0027B089002865
:1009B00000D000BF2F462C8A20480440F088044312
:1009C0002C82AC891E480440B08831890843718963
:1009D00008430443AC81AC8A1A480440B0890443FC
:1009E000AC8201A8FFF71AFE1748874202D104988B
:1009F000089001E003980890326891001923089A42
:100A00005A431046FFF7B8FB079064210798FFF799
:100A1000B3FB04012109642041430798411A069160
:100A200006990901084632306421FFF7A5FB00074B
:100A3000000F04432C8109B0F0BD0000FFCF00007F
:100A4000F3E90000FFFC000000380140CA05D20DA8
:100A5000828070470FB410B503A9044B044A029872
:100A600000F01AF810BC08BC04B01847890D00014A
:100A70006000002002E008C8121F08C1002AFAD155
:100A800070477047002001E001C1121F002AFBD10E
:100A9000704780F310887047FFB58FB00F4604464B
:100AA000002606E025280AD0129A11999047641C66
:100AB000761C20780028F5D1304613B0F0BD002513
:100AC0000121814A009500E00543641C2378084613
:100AD000203B98401042F7D120782E2815D10420D1
:100AE00005436078641C2A280AD101CF641C009059
:100AF0000BE000990A22514330394018641C0090E1
:100B00002078014630390929F3D920786C280ED095
:100B100004DC4C2813D06A2812D104E074280ED0CB
:100B20007A280DD10BE001204005054307E00121A3
:100B3000090562780D43824201D16D18641C641C62
:100B40002078692843D006DC0028B5D063280BD074
:100B5000642804D13BE073280FD075285DD0129A29
:100B600011999047761CADE03878694608720020EC
:100B7000487202A80190012003E03868019000202B
:100B8000C0433F1D69070CD5002500E06D1C00998E
:100B90008D420FDA8542F9DB0199495D0029F5D1D3
:100BA00008E0002500E06D1C8542FCDB0199495DF1
:100BB0000029F8D1761907E0019801990078491CBD
:100BC0000191129A119990476D1EF5D27AE000209A
:100BD00001900A216802400F0E91022809D001CF2E
:100BE000C11700290ADA0A460021404291412D220C
:100BF00007E0FF1DFF08FF0003CFF2E72A0504D539
:100C00002B226B461A72012203E0EA070ED0202243
:100C1000F7E70C920BAA0B9218E00A200E90002125
:100C20006802400F0191022802D001CF0022F0E7B4
:100C3000FF1DFF08FF0003CFF8E7019B0E9AFFF7A7
:100C4000D5FA0B9B5B1E30320B931A7002460A4397
:100C5000F3D10B9803A9081A20300190680701D43A
:100C60000120009000990198814203DD0846019916
:100C7000401A00E000200025009006E002A8129A29
:100C8000405D119990476D1C761C0C988542F5DBF0
:100C900004E0129A302011999047761C0099481E62
:100CA00000900029F5DC08E00B980B990078491CAE
:100CB0000B91129A11999047761C0199481E019048
:100CC0000029F1DC641CF4E60928010010B50121BB
:100CD000074800F079F84021064800F075F8012136
:100CE000034800F009F84021024800F005F810BD63
:100CF000000C01400008014070B504460D4629462D
:100D00002046FFF7A5FB70BD70B504460D46294689
:100D10002046FFF79FFB70BD00B58BB00121082076
:100D2000FFF76CFC01218803FFF768FC05A8FFF7BB
:100D300081FB402005900220069004200A9005A91E
:100D40000F48FFF7F3FA8020059004200A9005A9C8
:100D50000B48FFF7EBFAE1204002019000216846C2
:100D600001814181818101820C21C18101A9054854
:100D7000FFF712FE01210348FFF7EEFD0BB000BDA7
:100D8000000C01400038014070B504460D460A2CA5
:100D90000AD10D210B48FFF759FE00BF80210948F9
:100DA000FFF7EAFD0028F9D0E1B20648FFF74EFE52
:100DB00000BF80210348FFF7DFFD0028F9D020465F
:100DC00070BD00000038014030B587B004460D46C4
:100DD0000E48844204D101210420FFF70FFC09E0F2
:100DE0000B48844204D101210820FFF707FC01E0F1
:100DF00007B030BD01A8FFF71DFB0195012002904F
:100E000001A92046FFF792FA00BFF1E70008014070
:100E1000000C0140FFF700FDFFF77EFF0AA0FFF77F
:100E200019FE14A0FFF716FE1C4801681CA0FFF76E
:100E300011FE22A0FFF70EFEFFF748FFFFF73AFA78
:100E400000F0F6FC00BFFEE70A3D3D3D3D3D3D3D67
:100E50003D3D3D3D3D3D3D3D3D3D3D3D3D3D3D3DC2
:100E60003D3D3D3D3D3D3D3D3D3D3D3D3D3D3D3DB2
:100E70003D0A0000204E3332574230333120467253
:100E8000656552544F53202B2055415254202B203E
:100E90004C45442064656D6F0A000000000000208E
:100EA0002053797374656D436F7265436C6F636B28
:100EB000203D20256C7520487A0A00003D3D3D3DCF
:100EC0003D3D3D3D3D3D3D3D3D3D3D3D3D3D3D3D52
:100ED0003D3D3D3D3D3D3D3D3D3D3D3D3D3D3D3D42
:100EE0003D3D3D3D0A000000F8B505460E46174859
:100EF000076817480068001D00F096FB681C002872
:100F000008D1002E06D012480168091D114800F0D2
:100F1000CAFB1AE07C190E4800684460BC4207D244
:100F20000B480168091D0C48006800F0A1FB0CE0AB
:100F300007480168091D0948006800F099FB084846
:100F40000068844201D206480460F8BD1800002001
:100F500004000020740100200C0000200800002084
:100F60003400002010B5044600F0AAFB22480068B7
:100F7000401C2149086021480068002808D11F480A
:100F800004600846006801280ED100F07DF90BE0EE
:100F90001B480068002807D118480068C06AE16A49
:100FA000884201D81548046016480068401C15495D
:100FB00008600846006860641349E06A096888426E
:100FC00002D91149E06A08601422E16A51430F4ACC
:100FD0008818211D00F067FB00F080FB08480068BE
:100FE000002807D005480068C06AE16A884201D23B
:100FF00000F0C8FB10BD0000140000200400002019
:1010000020000020300000201C000020980000205C
:1010100010B516E000F054FB0C48C068C468201DF1
:1010200000F002FB0A480068401E094908600948B0
:101030000068401E0749086000F050FB204600F0A1
:1010400061F8044800680028E4D110BD6001002068
:10105000140000201000002070B504460D46206CDE
:1010600000280ED0216CE0684018E0606168E068FC
:10107000884201D32068E0602846226CE168FFF7CF
:1010800091F870BDF8B504460F4615460020009053
:10109000A66B206C002809D1206800282ED160683A
:1010A00000F02AFF00900020606027E0002D0FD1A3
:1010B0003946226CA068FFF775F8216CA0684018CB
:1010C000A0606168A068884218D32068A06015E01D
:1010D0003946226CE068FFF765F8216CE068401A39
:1010E000E0602168E068884203D2216C6068401AA1
:1010F000E060022D02D1002E00D0761E701CA0638D
:101100000098F8BD10B50446206B00F0FBFA2046AD
:1011100000F0F8FA10BD000030B501235B0317485A
:101120004407640F002C05D0C01DC008C000134C3C
:10113000041B1B1B0246124C22600024104D6C60E5
:10114000D0180838C008C0000E4C206000240D4D97
:101150002D686C600B4D2D682C601146441A4C6054
:10116000084C24680C60084D4C682C60074D4C6896
:101170002C600124E407064D2C6030BD880100205E
:10118000440000204C0000205400002050000020AB
:101190005800002000BFFFF73BFF0348006801280C
:1011A000F9D900F0EFFAF6E798000020FFB581B01A
:1011B00006460D4617460A9C002D01D1246000E02A
:1011C0002760E66325640121204600F0F3FB4C21F3
:1011D0000498085505B0F0BDFFB581B00F460A9ED2
:1011E0000C9C039A9100A522206BFEF7EDFF216B6A
:1011F0000398401E8000081800900098C008C000A6
:10120000009000984007400F002801D1012000E025
:101210000020002802D172B600BFFEE7002508E0DA
:10122000795D204634304155785D002800D102E0D8
:101230006D1C102DF4D300BF002143200155072E53
:1012400000D30626E662E66400202065201D00F03B
:101250000CFA2046183000F008FA24610720801BA1
:10126000A061646200206065002158200155049A45
:101270000199009800F0A6F920600B98002801D091
:101280000B98046005B0F0BD10B5002406E01421F1
:1012900061430E4A881800F0DBF9641C072CF6D372
:1012A0000B4800F0D5F90B4800F0D2F90A4800F0DD
:1012B000CFF90A4800F0CCF9094800F0C9F9044810
:1012C0000849086003480849086010BD98000020DC
:1012D00024010020380100204C0100206001002082
:1012E00074010020080000200C00002010B5014609
:1012F000164800E0006803688B42FBD3024643684F
:101300009B188B4204D143684C681B19436001460B
:101310000A464B689B180468A34211D10C4C036821
:101320002468A34208D04B68046864681B194B60AA
:1013300003681B680B6005E0054B1B680B6001E050
:1013400003680B60884200D0016010BD440000209B
:101350004C00002070B5054600F0B2F9A86B0028DB
:1013600001D1012400E0002400F0B8F9204670BD4E
:1013700070B5054600F0A4F9A86BE96B884201D16D
:10138000012400E0002400F0A9F9204670BD00000F
:101390000B4909680968002901D1012100E00021F9
:1013A000002904D00021C943064A116006E004491F
:1013B0000968C968C868034A41681160704700003D
:1013C000080000203400002010B500200749086103
:1013D00088617D21C90006480068FEF7CDFE401EE9
:1013E000024948610720086110BD000000E000E0EC
:1013F0000000002007480068401C002801D101209F
:1014000000E00020002802D172B600BFFEE772B6ED
:1014100000BFFEE74000002070B5044600F050F920
:101420004520055713E0606A002801D1012000E043
:101430000020002808D12046243000F0A1FD00281B
:1014400003D000F0D9F900E003E0681E45B2002D9A
:10145000E9DC00BF0021C9434520015500F03EF9F9
:1014600000F02EF94420055713E02069002801D12F
:10147000012000E0002000280AD12046103000F0B2
:101480007FFD002801D000F0B7F9681E45B200E0EA
:1014900001E0002DE9DC00BF0021C94344200155D3
:1014A00000F01CF970BD0000F8B504460020009063
:1014B00000F0F4F93E480068002801D1FFF72CFE47
:1014C0003C4800682040002861D1002C15D0083429
:1014D0006007400F002810D06007400F0821081A4D
:1014E00004196007400F002801D1012000E000200E
:1014F000002802D172B600BFFEE7002C47D02E486C
:101500000068844243D82D4E3046056801E02E46DF
:101510002D686868A04202D228680028F7D12448C4
:101520000068854233D03068083000902868306009
:101530006868001B102813D92F197807400F00285E
:1015400001D1012000E00020002802D172B600BFC6
:10155000FEE76868001B78606C603846FFF7C6FEDF
:10156000154968680968081A134908600846006840
:1015700013490968884203D20F480068104908607F
:101580000C4968680968084368600020286000F01A
:101590003BFD00984007400F002801D1012000E0EA
:1015A0000020002802D172B600BFFEE70098F8BD07
:1015B0004C00002058000020500000204400002073
:1015C00054000020001F01231B060360001F016060
:1015D000001F034B0360143802602038704700007E
:1015E000F513000170B5D2B00024002500BFEFF361
:1015F00010800646FF21453101A8FEF7ECFD01AC45
:1016000001349822074901A8FEF7CCFD0120FFF71D
:1016100040FAA04705463046FFF73BFA284652B04D
:1016200070BD00003822000101460A694B688868D5
:1016300098608B68486858605068884201D1886813
:101640005060002008611068401E106010687047EC
:101650000146083141600021C943816001460831DB
:10166000C160016100210160704700210161704784
:1016700010B502460B685C1C002C01D1106907E014
:101680001046083000E04068446824689C42FAD95B
:1016900044684C604C68A160886041600A611468CD
:1016A000641C146010BD42684A6093688B60936844
:1016B00059609160086103685B1C0360704700001B
:1016C00072B605480068401C03490860BFF34F8F9D
:1016D000BFF36F8F7047000040000020084800688B
:1016E000002802D172B600BFFEE705480068401E20
:1016F0000349086008460068002800D162B67047B8
:101700004000002070B506463546002E35D0083D15
:101710002C461A49606809680840002801D0012059
:1017200000E00020002802D172B600BFFEE720686A
:10173000002801D1012000E00020002802D172B66B
:1017400000BFFEE70D49606809680840002814D012
:101750002068002811D109496068096888436060E1
:1017600000F09CF806496068096840180449086060
:101770002046FFF7BBFD00F047FC70BD580000207D
:10178000500000200120000703494860BFF34F8F3D
:10179000BFF36F8F7047000000ED00E070B50446A6
:1017A0000025002C14D00D480068002801D101202C
:1017B00000E00020002802D172B600BFFEE700F072
:1017C0006DF800212046FFF78FFB00F01DFC054659
:1017D000002D01D1FFF7D6FF70BD00003C000020B6
:1017E00003490968016003490968416070470000C6
:1017F0002C000020180000200120014908607047DB
:101800002800002070B504460D46002C02D172B6A7
:1018100000BFFEE70548016818312046FFF728FFA2
:1018200001212846FFF760FB70BD00000400002086
:101830001CB5134800210B4680220091019011A194
:10184000124800F07BFA0446012C0DD172B600203C
:10185000C0430F49086001200E49086000200E496E
:10186000086000F063F80AE0601C002801D0012045
:1018700000E00020002802D172B600BFFEE71CBDC8
:101880003800002049444C4500000000951100013B
:1018900034000020200000201800002002480068CA
:1018A000401C0149086070473C0000201A4800684D
:1018B000002803D00120194908602CE000201749B6
:1018C00008601748016805E0002902D172B600BF20
:1018D000FEE7491E14204843124A1058002801D13F
:1018E000012000E000200028EED114224A430D4BD5
:1018F000D0184268526842600246083243689342F8
:1019000002D14268526842604268D268064B1A604F
:101910000348016000BF70473C0000202800002001
:101920001C000020980000200400002010B50B4887
:10193000006AFF2109040843084908620846006A52
:10194000FF210906084305490862FFF73DFD002015
:1019500003490860FEF7C6FB002010BD00ED00E063
:1019600040000020F7B582B005460E46002D01D09C
:10197000012000E00020002802D172B600BFFEE77F
:10198000002E01D1002701E02F4677433846503022
:10199000FFF78AFD0446002C09D020465030019004
:1019A000009431462846049B019AFFF7FFFB20462E
:1019B00005B0F0BD70B505460E462C46002C02D190
:1019C00072B600BFFEE7FFF77BFE216CE06B484379
:1019D0002168401860600020A0632068A060E06B70
:1019E000401E216C484321684018E0600021C94333
:1019F0004420015545200155002E10D120690028B2
:101A000001D1012000E00020002810D12046103034
:101A100000F0B6FA00280AD0FFF7B4FE07E020462F
:101A20001030FFF715FE20462430FFF711FEFFF7B8
:101A300055FE012070BDFFB583B006461D4600204F
:101A400002903446002C02D172B600BFFEE7049823
:101A5000002802D1206C002801D1012000E00020E4
:101A6000002802D172B600BFFEE7022D02D1E06B62
:101A7000012801D1012000E00020002802D172B627
:101A800000BFFEE700F088F9002802D10598002881
:101A900001D1012000E00020002802D172B600BF71
:101AA000FEE700BFFFF70CFEA06BE16B884201D39D
:101AB000022D1FD12A4620460499FFF7E3FA074674
:101AC000606A002801D1012000E00020002808D130
:101AD0002046243000F054FA002806D0FFF752FECA
:101AE00003E0002F01D0FFF74DFEFFF7F7FD0120C7
:101AF00007B0F0BD0598002803D1FFF7EFFD0020E7
:101B0000F6E70298002804D16846FFF769FE012035
:101B10000290FFF7E3FDFFF7C1FEFFF7D1FD44217F
:101B20000857401C002802D10021442001554521BE
:101B30000857401C002802D1002145200155FFF71D
:101B4000CDFD05A9684600F0BFF8002819D1204650
:101B5000FFF70EFC00280ED0204610300599FFF745
:101B600051FE2046FFF758FC00F04EFA002899D1AC
:101B7000FFF708FE96E72046FFF74EFC00F044FA18
:101B800090E72046FFF748FC00F03EFA0020AFE760
:101B9000F7B584B005460E46002003902C46002C75
:101BA00002D172B600BFFEE7002E02D1206C0028E1
:101BB00001D1012000E00020002802D172B600BF50
:101BC000FEE700F0E9F8002802D10698002801D1CC
:101BD000012000E00020002802D172B600BFFEE71D
:101BE00000BFFFF76DFDA76B002F1AD031462046CE
:101BF000FFF732FA781EA0632069002801D1012086
:101C000000E00020002807D12046103000F0B8F98D
:101C1000002801D0FFF7B6FDFFF760FD012007B0F7
:101C2000F0BD0698002803D1FFF758FD0020F6E725
:101C30000398002804D101A8FFF7D2FD01200390EA
:101C4000FFF74CFDFFF72AFEFFF73AFD4421085746
:101C5000401C002802D1002144200155452108578D
:101C6000401C002802D1002145200155FFF736FD18
:101C700006A901A800F028F8002819D12046FFF78E
:101C800069FB00280ED0204624300699FFF7BAFDE4
:101C90002046FFF7C1FB00F0B7F90028A1D1FFF7FC
:101CA00071FD9EE72046FFF7B7FB00F0ADF998E71E
:101CB0002046FFF7B1FB00F0A7F92046FFF74AFBEB
:101CC00000288ED00020AAE770B505460C46002DEE
:101CD00002D172B600BFFEE7002C02D172B600BF7F
:101CE000FEE7FFF7EDFC134802686868131A2068E6
:101CF000401C002801D1002617E00F492868096818
:101D0000884204D06868904201D801260DE020681E
:101D1000984207D92068C01A20602846FFF760FD66
:101D2000002602E0002020600126FFF7D7FC3046A5
:101D300070BD0000180000202C000020FFB585B009
:101D40001746B800FFF7B0FB0646002E0BD05C200C
:101D5000FFF7AAFB0446002C01D0266304E03046BE
:101D6000FFF7D0FC00E00024002C10D000220F99D7
:101D70000E986B4613C303923A46089B0699059842
:101D8000FFF72AFA2046FFF7EDF8012501E00025CC
:101D9000ED43284609B0F0BD06490968002901D184
:101DA000012006E004490968002901D1022000E071
:101DB00000207047200000203C000020F8B50020E3
:101DC000009042480068002872D141480068451CD4
:101DD0003F480560002D1CD13E480068006800287F
:101DE00001D1012000E00020002802D172B600BF1E
:101DF000FEE73848076838480068364908603648C2
:101E0000076036480068401C34490860FFF7C0FA94
:101E100000BF3348006885423DD300BF2D480068AD
:101E20000068002801D1012000E00020002804D033
:101E30000020C0432A4908602CE026480068C0689A
:101E4000C4686668B54202D22548066022E0201DBB
:101E5000FFF7EAFBA06A002803D020461830FFF7FE
:101E6000E3FB2049E06A0968884202D91D49E06A1B
:101E700008601422E16A51431B4A8818211DFFF7AC
:101E800012FC1A49E06A0968C96A8842C6D301206F
:101E90000090C3E700BF15480068C06A142148439A
:101EA00011490858012801D90120009005E0FFE7F9
:101EB0000F480068401C0E4908600E480068002862
:101EC00001D0012000900098F8BD00003C000020E7
:101ED00018000020080000200C0000202C0000202A
:101EE000340000201C000020980000200400002086
:101EF000240000202800002070B505462C4600264E
:101F0000002D35D01B480068844201D1012000E03B
:101F10000020002802D172B600BFFEE7206D002825
:101F200002D172B600BFFEE7206D401E2065E16C55
:101F3000E06A88421CD0206D002819D1201DFFF7CF
:101F400073FBE06CE0620721E06A081AA0610A49AD
:101F5000E06A0968884202D90749E06A08601422E9
:101F6000E16A5143054A8818211DFFF79CFB0126B1
:101F7000304670BD040000201C00002098000020A6
:101F800070B50646F068C468002C02D172B600BF76
:101F9000FEE720461830FFF747FB15480068002889
:101FA00013D1201DFFF740FB1249E06A09688842FF
:101FB00002D91049E06A08601422E16A51430E4ACE
:101FC0008818211DFFF76FFB04E0214618310B48EC
:101FD000FFF769FB0A49E06A0968C96A884204D9BF
:101FE000012501200749086000E00025284670BD52
:101FF0003C0000201C000020980000204C01002024
:10200000040000202800002070B50024002632487B
:102010000068002802D172B600BFFEE7FFF750FB50
:102020002D480068401E2C490860084600680028BA
:102030004DD12A480068002849D022E02848C068CD
:10204000C46820461830FFF7EFFA201DFFF7ECFABE
:102050002449E06A0968884202D92249E06A086096
:102060001422E16A5143204A8818211DFFF71BFB07
:102070001E49E06A0968C96A884202D301201C49E6
:10208000086017480068002801D1012000E0002006
:102090000028D3D0002C01D0FFF77AF91548056845
:1020A000002D0DD000BFFFF789FE002802D00120CF
:1020B0000F4908606D1E002DF5D100200D49086004
:1020C0000B480068002802D00126FFF75BFBFFF7F2
:1020D00005FB304670BD00003C00002014000020CD
:1020E0004C0100201C00002098000020040000206B
:1020F000280000202400002040BA7047C0BA704772
:102100000138FDD170470000F7B50325AD06286AF8
:1021100082B016460C46400840002862286A022118
:1021200008432862286A8007FCD46620686001277B
:102130002F61A86AC005FCD5992068602F61A86A44
:10214000C005FCD5FF209130FFF7DAFFFF230133F4
:10215000AB626846EF60352169602F61A96AC905E5
:10216000FCD5AB62A969EF60C9B205226A602F6134
:10217000AA6AD205FCD5AB62AA690902D2B21143A0
:102180000180C80702D0032005B0F0BDAB626869CA
:10219000FF210831884368616869C91E0843686186
:1021A00002980002483068600820A860EE602F6145
:1021B000A86AC005FCD5FF200130A8620023F61CE8
:1021C000B0080ED0B2081148006899006054060AA1
:1021D00009194E70060C000E8E705B1CC8709A4276
:1021E000F1D8FF200130A8626869FF2108318843D7
:1021F0006861686938436861286A800880002862DD
:10220000286A38432862002005B0F0BD8000000C29
:10221000032080064169FF220832914341614269EF
:1022200001210A434261026A920892000262026A34
:102230000A43026270470000002003218906096AF0
:10224000490849000322920611621146096A0222D6
:10225000114303229206116200BF03218906096A15
:10226000022211400229F8D0D10103229206916284
:102270000321D1609F2151600121116100BF032121
:102280008906896AFF22013211409142F7D1032267
:1022900092069162114688694969FF22083291438A
:1022A000032292065161114649690122114303221A
:1022B000920651611146096A890889001162114626
:1022C000096A01221143032292061162704700003D
:1022D00000000000010203040000010201000000F0
:1022E0000000000002000000000000000C230001BC
:1022F0000000002064000000740A00017023000147
:102300006400002024290000840A00010090D0030A
:1023100000000000000000000000000000000000BD
:1023200000000000000000000000000000000000AD
:10233000000000000000000000000000000000009D
:10234000000000000000000000000000AAAAAAAAE5
:10235000000000000000000000000000000000007D
:10236000000000000000000000000000000000006D
:04000005010000C135
:00000001FF
